:1000000011C029C028C028C026C025C024C023C0D4
:1000100022C021C03CC04BC062C073C07AC08AC03D
:10002000A0C0B0C011241FBECFE9CDBF10E0A0E634
:10003000B0E0E0EEF2E002C005900D92A236B1070A
:10004000D9F710E0A2E6B0E001C01D92AB36B107CF
:10005000E1F7CBD043C1D4CF1F920F920FB60F92CE
:1000600011248F939F93EF93FF9384EC82BF87B308
:10007000807F87BB88B3807F88BBE0916400F0E01D
:10008000E830F10508F086C0E65FFF4F09948091E3
:100090006200813049F080916200833029F08091C4
:1000A0006200853009F076C087B3836068C08091B4
:1000B0006200823089F080916200833069F0809123
:1000C0006200843049F080916200853029F080918F
:1000D0006200863009F05EC087B383600FC08091F4
:1000E0006200843049F080916200853029F080916F
:1000F0006200863009F04EC087B3866087BBC19A24
:1001000049C080916200863009F044C087B38660A0
:100110000EC080916300813041F080916300833094
:1001200021F0809163008530A9F587B38C6087BB8F
:10013000C29A30C080916300823081F08091630068
:10014000833061F080916300843041F080916300DE
:10015000853021F0809163008630E1F487B38C60B4
:1001600017C080916300843041F080916300853036
:1001700021F080916300863069F487B3896087BB82
:10018000C09A08C080916300863021F487B38960EB
:1001900087BBC39A809164008F5F809364008091D5
:1001A0006400883010F010926400809160008F5FCE
:1001B0008093600080916000873070F091E09093B0
:1001C0006000809161008F5F809361008091610089
:1001D000873010F090936100FF91EF919F918F9184
:1001E0000F900FBE0F901F90189585B5836085BD49
:1001F00085B58D7F85BD81E080936200809363002B
:1002000083B7826083BF89B7826089BF7894B499CD
:100210000DC0109262001092630080916000809384
:1002200068008091610080936700F1CF8091620047
:10023000882369F710926A00109269002DC080919E
:10024000600080936200809161008093630010924F
:100250006600109265000CC08FE599E00197F1F7F8
:1002600000C000004F5F5F4F5093660040936500F1
:100270002091690030916A00C901B9011DD04091F7
:100280006500509166004817590730F32F5F3F4FC4
:1002900030936A00209369008091690090916A0010
:1002A0008431910560F280916800809362008091B2
:1002B000670080936300ABCF5527002480FF02C006
:1002C000060E571F660F771F6115710521F0969571
:1002D0008795009799F7952F802D0895F894FFCF73
:0202E00001011A
:00000001FF
